:1000000002003000000000000000000000000000BE
:1000100000000000000000000000000000000000E0
:1000200000000000000000000000000000000000D0
:100030001207DDC2A07920770009E4B960F9755094
:100040005075515075525075535075546A75556AB4
:1000500075566A75576A75585A75595A755A5A7548
:100060005B5A053875815F758955C2A1D2081203A4
:1000700036F53FF541754000D20A120A48120A1CB3
:10008000D2011208B8C2011208B8C2241200AAC2D2
:10009000A0432030A21072144006753B1802065788
:1000A000201004D202C29202065CC2A1C29220A712
:1000B00008B29120A7030200C0D224D202120E88F7
:1000C000D29220A708B29120A7030200D4D224C262
:1000D00002120E88227912E37914C295E3D2957A3E
:1000E000DC20A62BDAFBC20C12034D7B0020A61FDE
:1000F00020A61C20A61920A616DAF220A611DBEDF8
:10010000D2A1D20812034DDDE4C2A07DFF80DE2023
:10011000240211AA753B00C221C220C222C29379D7
:1001200004E37E01A2E3920F5477F520E4A2029249
:10013000E1A20192E02450F5472408F8E6A2E092FB
:100140002320061520050920040302064402092283
:100150002004030208680209407D1E200F027D036F
:1001600020050B300403020179C221020369200437
:10017000030205ECC2200203EC790EE3B400057E15
:100180000A020369B40105D2200203ECB40208D2CA
:10019000931201EE0201B8B40303020218B4041072
:1001A000D29379087409F3E4790AF309F30201B8E8
:1001B000B40505D221020369C207120886E53B6037
:1001C00002D2071206ADD203C293E4F91206E0127E
:1001D00006E01206E01206E0790EE5391206E0E5C7
:1001E000381206E0E53A1206E075815F01D5120784
:1001F000E31202BA790874503023027428F3854B55
:10020000F0E54D0403030345F0790AF3790CE54C5E
:10021000440844104440F322790AE35403B4010330
:100220000202257402F5F0E3540CB404030202B494
:10023000740842F0E35430B420027410E354C0B4A4
:1002400080030202B4744045F0F3C22330E016D2BA
:10025000237906E3B4000D02025DB4FF0774503049
:1002600023027428F37908E3541FB4000D020273CB
:10027000B41F07740A3023027409F5F0E354E0B4A4
:100280000008020288B407027460B405030202B4D5
:10029000B406030202B445F0F37806E2A947F77802
:1002A00008E5472404F9E2F7780AE5472408F9E26B
:1002B000F702065C753BEC020657853945C2A11270
:1002C00008B87403120C7020D541E4B53B3D753974
:1002D0000275471F12048FE4B53B3012059AE4B54E
:1002E0003B2985304CC223E54CB40102D223754B27
:1002F00000754E2812059AE54BC2D79532500385FA
:10030000324BD54EEF85334D02030E753BE48545E8
:100310003922302305781AE203F222302305781AB5
:10032000E223F222E53930230323F53922E539307F
:10033000230303F539227F04E4AC905390F0A2A785
:100340003305900590DFF78C90C4F54122A2A1926D
:100350000FC2A171366540600B423F200A06C2946D
:10036000D294D20AA20F92A1227906E3F539712420
:100370007908E3F5381207E312048F7912E3791054
:10038000781CE538F271127818E4FAFB7482209038
:1003900002748AF2781E20A708753B50711B020771
:1003A000D620A50F20A43EDAF8DBF6711B1207DD7C
:1003B0000204DEE2302111F5F0E3B5F0030203C9D7
:1003C000753BFC711B0207D6F37F0620A5E5DFFB1A
:1003D0007F16DFFE20A40E753B7020A703753BA09F
:1003E000711B0207D6711B120767808F7906E3F530
:1003F000397908E3F5381207E3302306753B2C0200
:10040000068512048FE539C297B42C005005C296B8
:1004100002041FB43D005005C29602041FD2967913
:1004200012E37910781CE538F27818E4FAFBD20C64
:1004300074A220900274AAA22092E0F2781EE32017
:10044000A706753B500207D620A50D20A43EDAEF83
:10045000DBED1207DD0204DEF2E37FE620A511DF0B
:10046000FB1207DD753B3020A703753B5002068564
:10047000F2E37F0620A5F9DFFB7F2EDFFE20A40C30
:10048000753B7020A703753B980207D602076712D9
:1004900006E8C2A130A01A200D111206347B8F7A13
:1004A0000020A415DAFBDBF90204CE200E120204B0
:1004B000B9D2A0300D13120C6E7403120C70C20866
:1004C0002008F6E539781AF222120C6E80CCE4FA94
:1004D000FB20A4E5DAFBDBF9753B400207D6753B50
:1004E0000012059AE53B60030206857818E2541C69
:1004F000702DE530B53913E531209006B4010502C1
:1005000005286024753B4802068585303A753B68AE
:1005100020910685303C02068585303D02068530F7
:10052000E406753BE002068575420A12053C753B00
:100530007820D503753BA8C2D502068512059AE539
:100540003B600D200607A20F92A002065702068507
:10055000D209D20B120767E532B53803D2D522D5BE
:1005600042DA227E01754201B13CC2D5853238752E
:10057000F00A0538E538B40B037538017E01754281
:1005800001B13C20D50A753BE0A20F92A0020657AC
:10059000C2D5D5F0DDA20F92A022AC8175812F7853
:1005A000187F02E4FAFB74C0F2781E20A708753B9E
:1005B000508C810207DD20A51120A42DDAEDDBEBA4
:1005C000DFE9753B588C810207DDE2C0E07F062041
:1005D000A5F8DFFB7F14DFFE20A40E753B7020A77B
:1005E00003753BA08C810207DD8C8122D222120789
:1005F000E3D20D120738C2A120A009C208D2A0740C
:1006000064120C70300807C2087403120C70B19A9F
:10061000E53B70717912E37910E530F539F3E53295
:10062000F538F3E531F3E533F3E534F3E535F3D2AB
:100630000B020767781EE539F2781AE53EF2781862
:100640007418F2221207E3D20D120738D2D5A2A1F4
:10065000920FC2A102065CD20702065EC207120612
:10066000AD120886D203C022C023E53E2022053009
:100670002302C313C0E0C03BC0207400C0E0740478
:10068000C0E00206C2D20702068CC2071206ADD233
:1006900003C03AC038E539302302C313C0E0C03B81
:1006A000C0207400C0E07404C0E00206C22250B54D
:1006B0003B0F1207DD7F0ADFFEE254406003753B0B
:1006C0005822C293E4F91206E01206E01206E0D2C4
:1006D000937F07F9D0E01206E0DFF975815F01D55D
:1006E000F30909220909E322E5472404F8E6541F27
:1006F000C395385005753BB8808B712DA847E6141B
:10070000C395395007753B207124C1857124E539A3
:1007100020010F653D601AC20D853D3E85393D02C1
:100720000733653C600BC20D853C3E85393C0207B2
:1007300033D20DE53802073875F00DE520F46590E9
:1007400054076015C20E300C03120C5FE520F45400
:10075000075390F84290C20C22D20E300C06200DA6
:1007600003120C5FC20C227818E230E506753BF4E8
:100770000207C430E706753B500207C430E610B1EB
:100780009AE53BB458030207C4753BB00207C43076
:10079000E206753B880207C020E41320E307C20B82
:1007A000200930C18A200B06753B800207C030E368
:1007B00006753B600207C0753B38200B03753B3064
:1007C000C20BDE0FC20BC209300602C185A20F9216
:1007D000A0C157C20922781874D0F2C18578187464
:1007E000D0F22220020A30101120110320000B2227
:1007F00030140720150320000122753B90200603CA
:100800000206570206851208B820D530D29074032C
:10081000120C7074487F1812084730E212753B08BA
:10082000209203753B108C90A20F92A00206577481
:1008300003120C701208B8D20820D5E1C2D58C90F2
:10084000A20F92A0227F057818F27B057A0020A4DF
:1008500013DAFBDBF9753B4074D0F28C90A20F9257
:10086000A0020657DFE3E2221207E3C2A1020E78DC
:100870008C90A20F92A0D20820D50302065CC2D5AC
:10088000753B280206571207DD853F23E522853D8B
:100890003E209104853C3E0054034223E230E602B0
:1008A000D21BA2A7921A30D50EA20F92A1753F00BB
:1008B000854140C20AC2D522C2D5A2A0920FD2A0C1
:1008C000120738AC90D29078187408F27F03E4FADB
:1008D000FB20A41820A415DAF8DBF6DFF4A20F92AF
:1008E000A08C90753B401207DD020657E220E2051E
:1008F000D2D5020921C290000000000000000000D3
:10090000309110753D00D2100000E230E21300007B
:10091000020921753C00D2120000E230E20300001F
:1009200000221207E3120A48120A1CD20D120738DD
:10093000C2A1C2081209BF12096512056302065C52
:1009400074FFF580F590F5A0F5B0F4F5F0F5A8F595
:10095000D0F588F589F598F58AF58CF58BF58D90AD
:1009600000000200007E0175420112053CC2D585DF
:100970003043E530B44B00744875F0684002C5F070
:1009800011457E01754201120E93C2D5853044C5D2
:10099000F011457E01754201120E93C2D5C530B5E6
:1009A000430A9544B4050122B4FB0A22F53D209187
:1009B00002F53CC53EA20F92A0753BE80206572007
:1009C000A706753B50020657A2A0920F20A007D29F
:1009D000A07447120C70781874D4F2E4FAFB20A4C7
:1009E00017DAFBDBF91207DD12059AE53B6003021B
:1009F0000A15753BD0020A1574D4F27BC47AA7207D
:100A0000A410DAFBDBF77B057AA630A40122DAFA20
:100A1000DBF6753BD8A20F92A0020657E4F58AF5E3
:100A20008CC28DFA7BA6D28C208D12DAFBDBF97B8F
:100A3000077AD1208D0F208D0CDAF8DBF4C28C758B
:100A40003BF0020657C28C22120ADD120A85120AF6
:100A500094120AD1D3120C12C3120C12E4F5F01244
:100A60000BBEF4F5F0120BBE7455F5F0F4120BBE8C
:100A7000C5F075F055120BBE120AA3120AA922790D
:100A800012F3791022517F120AA3120AA3120AAF9D
:100A9000120AAF22517F120AA3120AA9120AAF1238
:100AA0000AC022E4F30470FC22E414F370FC227FF9
:100AB00000E36F6006753BF80206570FBF00F22295
:100AC0007F001FE36F6006753BF8020657BF00F218
:100AD00022E4CC120B82CCB2E00360F622120B01AE
:100AE000120BE1120B2622E5F0F3E4E365F070014E
:100AF00022E4FF517FF3DFFDF3DFFD753BF80206D3
:100B000057D2937904747FF3E4E33340E47480F3C1
:100B1000E4E33350DC790675F0C051E775F0C85155
:100B2000E775F0F880C17480C5F0120B41C5F0C3C1
:100B30001350F5747FC5F0120B41C5F0D31340F587
:100B400022D2937900E5F01206E003B90EF9C293C0
:100B50007900E5F0F41206E003B90EF979FED293BC
:100B6000E5F0CF1206E46F706BCF03B90CF479FE99
:100B7000C293E5F0CF1206E4F46F7058CF03B90CBE
:100B8000F322EC7B107A10F3B2E003DAFA7A10F376
:100B9000B2E723DAFADBEE8CF07B107A10E365F033
:100BA0007032C5F0B2E003C5F0DAF27A10E365F016
:100BB0007022C5F0B2E723C5F0DAF2DBDE227F0057
:100BC000FCF3E5F0F3ECDFF9E36C7008E365F0703B
:100BD00003DFF522540F753BC86003753BC0020666
:100BE00057D2937900E91206E0B90EF9C293790061
:100BF000E91206E0B90EF9D29379FE1206E46970A3
:100C0000D3B90CF7C29379FE1206E46970C6B90C29
:100C1000F7227F20920FE44001F413F313200F0515
:100C200040F9020C2750F433F333200F0540F9024A
:100C30000C3450F4DFE47F2013CCE36C7096CC13BB
:100C4000200F0540F4020C4A50EF33CCE36C708463
:100C5000CC33200F0540F4020C5C50EFDFDA227F2A
:100C60001500DFFDD5F0F82275F064915F2274471E
:100C70009168D5E0FB22FFFFFFFFFFFFFFFFFFFFB3
:100E7000FFFFFFFFFFFFFFFFB2011208B8B2011230
:100E800008B8020870FFFFFFA291B39201020806A2
:100E9000FFFFFFFAABF07405120C70EA8BF002054D
:100EA0003CFFFFFFFFFFFFFFFFFFFFFFFFFFFFFF15
:100FF000FFFFFFFFFFFFFFFFFFFFFFFFFFFFFF60A0
:00000001FF
